:020000040000FA
:10000000250005046600670040000200140A060C83
:100010003000F002090A0C0A00080F0C3000030C33
:100020000600F002110A0008460440000600070915
:10003000010C06001B0A0000400006000709010C25
:100040000600220A0000400006000709010C060015
:10005000290A0000400006000709010C0600300ACA
:100060000000400006000709010C0600370A0000E6
:1000700040000600010C060007093E0A000040008F
:100080000600010C06000709450A000040000600B2
:10009000010C060007094C0A000040000600010C94
:1000A00006000709530A000040000600010C060084
:1000B0000709310C31000000010C06004000060069
:1000C000610A0000010C06000D09F1025C0A010C36
:1000D0000600400006006C0A0000010C06000D0935
:1000E000F102670A40000600010C06000709780AC1
:1000F000000040000600010C060007097F0A00000E
:1001000040000600010C06000709860A00004000B6
:100110000600010C060007098D0A000040000600D9
:10012000010C06000709940A46054000060007096D
:10013000010C06009B0A0000400006000709010CA4
:100140000600A20A0000400006000709010C060094
:10015000A90A0000400006000709010C0600B00AC9
:100160000000400006000709010C0600B70A000065
:1001700040000600010C06000709BE0A000040000E
:100180000600010C06000709C50A00004000060031
:10019000010C06000709CC0A000040000600010C13
:1001A00006000709D30A000040000600010C060003
:1001B00007090709DB0ADC0ADD0ADE0A300C310018
:1001C000010C060040000600E50A0000010C0600D4
:1001D0000D09F102E00A010C060040000600F00AD9
:1001E0000000010C06000D09F102EB0A40000600B8
:1001F000F90A0000010C0600070940000600010C86
:1002000006000709030B000040000600010C060071
:1002100007090A0B000040000600010C0600070950
:10022000110B000040000600010C06000709180B26
:0E023000000040000600010C06000709140A39
:021FFE00EB0FE7
:00000001FF
